:020000040000FA
:10000000EBEF03F01200FFFF04EF04F01200FFFF1C
:10001000FFFFFFFFFFFFFFFF0CEF04F01200FFFFE9
:10002000FFFFFFFFFFFFFFFFFFFF00000001776BF7
:100030001E0E716E0401400E096F200E0A6F040E31
:100040000B6F880E086F0401200E0E6F040E0F6FE9
:10005000400E0C6F1200550EA76EAA0EA76EA68258
:1000600012000401050E226F010E236F1200000121
:10007000756B040121510001755D20E275C000F02F
:10008000016A026A040122510024F36E2351012007
:10009000F46E24510220F86EF4CFF7FFF3CFF6FF91
:1000A0000800F5CF76F000017551EA6A250FE96E78
:1000B000040EEA2276C0EFFF752BDBD7F86A120038
:1000C000F00E04012217840EA66E0001756B040168
:1000D00021510001755D26E27551EA6A250FE96E2E
:1000E000040EEA22EFCF03F075C000F0016A026A45
:1000F000040122510024F36E23510120F46E245197
:100100000220F86EF4CFF7FFF3CFF6FF03C0F5FF40
:100110000C000F0E000175150F0801E19CDF0001B6
:10012000752BD5D71200940EA66E0001756B0401D5
:1001300021510001755D1EE27551006E016A060EC7
:10014000D89000360136E804FBE1026A01BE02687D
:10015000040122510024F36E23510120F46E245136
:100160000220F86EF4CFF7FFF3CFF6FF74DF000143
:10017000752BDDD7F86A1200A66A0001756B0401C1
:1001800021510001755D10E2040122510001752525
:10019000A96EA6807551EA6A250FE96E040EEA225F
:1001A000A8CFEFFF752BEBD712000001756B040190
:1001B00021510001755D15E20401225100017525F0
:1001C000A96E7551EA6A250FE96E040EEA22EF5016
:1001D000A86E040EA66E3FDFA6B2FED70001752BF7
:1001E000E6D71200C40EA66E0001756B0401215102
:1001F0000001755D21E27551EA6A250FE96E040E72
:10020000EA22EFCF03F075C000F0016A026A040130
:1002100022510024F36E23510120F46E2451022058
:10022000F86EF4CFF7FFF3CFF6FF03C0F5FF0C0035
:1002300012DF0001752BDAD7F86A1200060E0001F2
:100240007A5D03E36D50020B01E071D00001770588
:1002500011E104010CBF0DD00401400E096F400EE6
:10026000040108170401087D880E04010813000129
:10027000776B5DD0040108BF5AD00001756B040193
:100280002051FF0A34E0F80A2DE0020A26E0010AB4
:100290001FE0070A18E0010A11E0030A0AE0070A52
:1002A00008E0060A01E032D0DCDE0001040E756FC2
:1002B0002ED0DDDE050E0001752729D001DF0001FB
:1002C000010E756F24D02FDF0001010E756F1FD056
:1002D00053DF050E000175271AD067DF0001010EFC
:1002E000756F15D07FDF0001010E756F10D06D9610
:1002F0000001786B796B00017807000E795B0001D3
:100300007851791101E0F7D7FF0001D000D000014A
:10031000010E776F000175510AE075C00DF4400EB3
:1003200004010C1704010C7D880E04010C1312004B
:100330006C5002E0000E01D0010E00090BE0040138
:1003400000513C0BE842E8420D0802E10CD801D014
:1003500013D808D06C5002E0000E01D0010E040941
:1003600001E01AD812000001606B616B666B676B6D
:100370009EEC02F04AEF02F0020E0001605D0AE11D
:1003800068D8040100BD03D0C80E006F02D0880EEB
:10039000006F01D0C5D81200040E00017A5D0AE199
:1003A00012C46EFF6E50000803E2050E7A6F02D091
:1003B000030E7A6F000160050AE10BD8040104BD49
:1003C00003D0C80E046F02D0880E046F01D0A8D8E5
:1003D00012000001080E665D000E675903E266C058
:1003E00069F002D0080E696F69C005F46951006EAA
:1003F000016A0050665F0150675B180E646F040E5F
:10040000656F695125E000017BA310D062C0F6FF43
:1004100063C0F7FF0800F55064C0E9FF65C0EAFF5C
:10042000EF6E0001622B000E63230ED062C0E9FF65
:1004300063C0EAFFEF5064C0E9FF65C0EAFFEF6EFA
:100440000001622B000E6323642B65236907D9D753
:10045000120001C46AF000016A516625666F000E41
:100460006721676F180E626F040E636F6A5111E0A7
:1004700062C0E9FF63C0EAFFEF5064C0E9FF65C0F6
:10048000EAFFEF6E642B000E6523622B63236A077D
:10049000EDD71200000161510CE10401080E016F5B
:1004A000100E026F040E036F840E006F0401046FC0
:1004B00035D0040110AF22D0000166510401165D51
:1004C000000167510401175904E216C466F017C40D
:1004D00067F07FDF0001010E606F0401080E016FFD
:1004E000100E026F040E036F800E006F0401180ED1
:1004F000066F040E076FC80E046F10D00001020EC5
:10050000606F0401056BC80E046F0401080E016FD3
:10051000180E026F040E036FC80E006F6D98120064
:100520000001606B0401080E016F100E026F040ED3
:10053000036F880E006F0401046B12000401105158
:10054000600BE842E842E842E842E842000901E084
:1005500050D01151080A3FE0010A3BE00F0A0AE0BF
:10056000030A01E046D00001010E616F0001040E94
:100570007A6F3FD00001010E616F040113050AE19B
:100580000001A00E626F070E636F120E0001666F0E
:10059000676B1CD0020E135D0AE10001B20E626FA0
:1005A000070E636F200E0001666F676B0FD0030E9E
:1005B000135D0AE10001D20E626F070E636F040E35
:1005C0000001666F676B02D00001616B00017B83E5
:1005D00010D010D80ED00001010E616F00017C0E0A
:1005E000626F000E636F00017B930001010E666F66
:1005F00000D012000001010E616F12C47CF00401F2
:10060000125104E10001050E7A6F05D00001060EBB
:100610007A6F16EC00F01200080E6D6E6DBAFED700
:10062000686A110E696E0001020E7A6F120068503E
:10063000040B06E06950040B03E06D926994689422
:100640006850010B04E06950010B01E027D86850A5
:10065000100B09E06950100B06E0698468986D8200
:10066000A08A0300A19A6850200B09E06950200B72
:1006700006E070A003D090EC02F07090689A030E30
:1006800000017A5D01E209D06850080B06E069506C
:10069000080B03E098EC01F068961200686A7B0E84
:1006A000696E6E6A160E706E68A602D06896FCD7E8
:1006B0006D9890EC02F000017C6B0001030E7A6FE4
:1006C00012002A0EF66E000EF76E000EF86E000194
:1006D0000900F550706F0900F550716F03E1706704
:1006E00001D03DD00900F5506B6F0900F5506C6FDB
:1006F0000900F5506D6F09000900F550E96E090019
:10070000F550EA6E090009000900F5506E6F090006
:10071000F5506F6F09000900F6CF72F0F7CF73F054
:10072000F8CF74F06BC0F6FF6CC0F7FF6DC0F8FF38
:1007300000016E5302E16F5307E00900F550EE6EC1
:100740006E07F8E26F07F9D772C0F6FF73C0F7FFC4
:1007500074C0F8FF00017007000E715BBFD7120074
:10076000A66AFE0EA96EA680A8CF7FF0FF0E00013C
:100770007F5D02E1000E01D0010E006E8450080B77
:1007800001E0010E001402E000EF04F0140E6F6EA1
:100790000CEC03F017EC03F01EEC01F0FBD7120099
:1007A0001201000200000008D8040BFF0000000046
:1007B000000109022000010100803209040000024A
:1007C000000000000705010240000007058102400B
:1007D00000000403090413EE00F023EE00F0F86AB1
:1007E000059C61EC03F0B0EC03F0FDD71200FFFFB5
:1007F000FFFFFFFFFFFFFFFFFFFFFFFFFFFFFFFF09
:1008000052EF2AF01200FFFF1200FFFFFFFFFFFF71
:10081000FFFFFFFFFFFFFFFF1200FFFFFFFFFFFFD4
:10082000FFFFFFFFFFFFFFFFFFFF0100005500007C
:10083000CA01000024000000D9CFE6FFE1CFD9FFB4
:10084000E6520101CC6B7F0ECD6FCE69C70ECF6F24
:10085000926893689468DF6ADFCF10F0050EE76E48
:100860001018E8AE02D0E73402D0E750105C01E384
:100870007BD0DFCFE9FFEA6AE9BEEA68040ED890D0
:10088000E936EA36E806FBE1410EE926010EEA22E6
:10089000EF6ADFCFE9FFEA6AE9BEEA68040ED890A2
:1008A000E936EA36E806FBE1410EE926010EEA22C6
:1008B000EE52EF6ADFCFE9FFEA6AE9BEEA68040EAA
:1008C000D890E936EA36E806FBE1410EE926010E4A
:1008D000EA22020EE926000EEA22EF6ADFCFE9FFE4
:1008E000EA6AE9BEEA68040ED890E936EA36E80614
:1008F000FBE1410EE926010EEA22030EE926000E75
:10090000EA22010EEF6EDFCFE9FFEA6AE9BEEA688C
:10091000040ED890E936EA36E806FBE1410EE926F6
:10092000010EEA22040EE926000EEA22EE6AED6AC2
:10093000DFCFE9FFEA6AE9BEEA68040ED890E9363B
:10094000EA36E806FBE1410EE926010EEA22060E30
:10095000E926000EEA22EE6AED6ADFCFE6FF58ECE8
:1009600013F0E552DF2A78D7DF6ADFCF10F0050EEB
:10097000E76E1018E8AE02D0E73402D0E750105C02
:100980005AE2DFCFE9FFEA6AE9BEEA68050EEA0249
:10099000F3CFEAFFE902F3CFE9FFF450EA26910E24
:1009A000E926010EEA22EF6ADFCFE9FFEA6AE9BE33
:1009B000EA68050EEA02F3CFEAFFE902F3CFE9FFA6
:1009C000F450EA26910EE926010EEA22EE52EF6A71
:1009D000DFCFE9FFEA6AE9BEEA68050EEA02F3CF73
:1009E000EAFFE902F3CFE9FFF450EA26910EE92687
:1009F000010EEA22020EE926000EEA22010EEF6E37
:100A0000DFCFE9FFEA6AE9BEEA68050EEA02F3CF42
:100A1000EAFFE902F3CFE9FFF450EA26910EE92656
:100A2000010EEA22030EE926000EEA22010EEE6E06
:100A3000ED6ADF2A9AD7E552E552E7CFD9FF1200D7
:100A4000060E0101F85D05E36D50020B01E0120096
:100A500001D81200D9CFE6FFE1CFD9FF050EE1267C
:100A6000400EE66E010EE66E010EE66E95EC26F087
:100A7000E552E552E552000901E1E8D00101006BC1
:100A800001010151FF0A01E1A8D0960A01E1A2D0BB
:100A9000010A01E19CD00D0A01E196D0010A01E1B1
:100AA00090D0070A01E187D0010A01E17ED0030A54
:100AB00076E0010A6EE03C0A66E0030A5EE0010AA5
:100AC00056E0030A4EE0070A49E0020A44E00F0A32
:100AD0003FE0010A3AE0030A35E0330A30E0010A58
:100AE0002BE0340A26E0070A21E00D0A1CE00B0A7D
:100AF00018E0030A14E0010A10E0500A01E08FD068
:100B000001010A0E036F0101020E046F01011C0EA8
:100B1000056F0101050E006F88D0F3D886D09DD9EE
:100B200084D093DA82D0EDEC09F07FD0F0EC0BF0BA
:100B30007CD0F8EC0CF079D002EC0EF076D05AECC8
:100B40000EF073D0B8EC0FF070D0B8EC0FF06DD0A1
:100B5000FCEC10F06AD09AEC11F067D038EC12F08F
:100B600064D0010EE66E6EEC15F0E5525ED0020E1A
:100B7000E66E6EEC15F0E55258D0030EE66E6EECA4
:100B800015F0E55252D0040EE66E6EEC15F0E5520B
:100B90004CD0010EE66EFAEC1AF0E55246D0020E89
:100BA000E66EFAEC1AF0E55240D0030EE66EFAEC6F
:100BB0001AF0E5523AD0040EE66EFAEC1AF0E5525D
:100BC00034D013EC1EF031D04DEC1EF02ED06CEC76
:100BD00020F02BD0BFEC20F028D06D96010EDB6A00
:100BE000020EDB6A010EDB06DBCF10F0020E01E223
:100BF000DB06DBCF11F01050111001E0F3D7FA0E35
:100C0000E66EE66A93EC21F0E552E552FA0EE66EE6
:100C1000E66A93EC21F0E552E552FF0006D00101AF
:100C200001690101100E006F00D0010100510EE0BA
:100C300004010CBF0BD000C1E6FF010EE66E010EF1
:100C4000E66E5BEC26F0E552E552E5520101D70570
:100C500002E114EC0BF00101520505E1010EE66E14
:100C6000BEEC19F0E5520101620505E1020EE66EE7
:100C7000BEEC19F0E5520101720505E1030EE66EC6
:100C8000BEEC19F0E5520101820505E1040EE66EA5
:100C9000BEEC19F0E5520101965105E0010EE66E39
:100CA00050EC1DF0E55201019B5105E0020EE66E8D
:100CB00050EC1DF0E5520101A05105E0030EE66E77
:100CC00050EC1DF0E5520101A55105E0040EE66E61
:100CD00050EC1DF0E5520101D90502E189EC1EF04E
:100CE0000101E30502E1A6EC1FF0F56E050EE15CE3
:100CF00002E2E16AE552E16EF550E552E7CFD9FF35
:100D0000120001010251070A01E192D0010A01E13A
:100D100080D0030A6CE0010A5BE0070A52E0010A96
:100D200035E0130A1EE0100A0AE0010A01E091D042
:100D30000101CD519212CE519312CF5156D0035191
:100D40000101CD15926E010104510101CE15936E82
:100D5000010105510101CF15946E010106B112D0B8
:100D600013D003510101CD15926E0101045101010F
:100D7000CE15936E010105510101CF15946E01014D
:100D800006A102D0F19E65D0F18E63D0035101011E
:100D9000CD15106ECD1D89141010896E01010451FE
:100DA0000101CE15106ECE1D8A1410108A6E01013D
:100DB00005510101CF15106ECF1D8B1410108B6ED5
:100DC00048D080CF03F181CF04F182CF05F141D02B
:100DD00003510101CD159212010104510101CE15FB
:100DE0009312010105510101CF15941232D0035124
:100DF0000101CD15E81C9216010104510101CE1527
:100E0000E81C9316010105510101CF15E81C941649
:100E100020D003510101CD158912010104510101B6
:100E2000CE158A12010105510101CF158B1211D087
:100E300003510101CD15E81C89160101045101017E
:100E4000CE15E81C8A16010105510101CF15E81CD9
:100E50008B160101100E006F1200D9CFE6FFE1CF13
:100E6000D9FFE65201010251030A01E1DFD0010A74
:100E700001E1C8D0030A0EE0010A01E0DED0C26A37
:100E80000F0EC16E0101D051CD13D151CE13D06BD5
:100E9000D16BD3D0C26AAA0EC06E03510A0A01E117
:100EA00091D0030A01E17ED0010A6CE00F0A5AE0FA
:100EB000010A49E0030A3EE0010A32E0070A26E09F
:100EC000010A1AE0030A0FE0010A01E08AD00F0EBE
:100ED000C16ED00E0101CD152F09CD6FE00ECE15DC
:100EE0001F09CE6F7ED092800101D081D00ECD152A
:100EF0002E09CD6F0E0E74D0030E92120101D01385
:100F0000D00ECD152C09CD6F0D0E6AD0070E9212A2
:100F10000101D013D00ECD152809CD6F0C0E60D075
:100F20000F0E92120101D013D00ECD152009CD6FF6
:100F30000B0E56D02F0E92120101D013D00ECD15EC
:100F4000CD6F0A0E4DD02F0E92120101D013D00E8C
:100F5000CD15CD6F9384D185E00ECE151B09CE6FD4
:100F6000060E3ED02F0E92120101D013D00ECD15D9
:100F7000CD6F0C0E9312D113E00ECE151309CE6F68
:100F8000050E2ED02F0E92120101D013D00ECD15CA
:100F9000CD6F0E0E9312D113E00ECE151109CE6F48
:100FA000040E1ED02F0E92120101D013D00ECD15BB
:100FB000CD6F1E0E9312D113E00ECE150109CE6F28
:100FC000030E0ED02F0E92120101D013D00ECD15AC
:100FD000CD6F1F0E9312D113E00ECE15CE6F020E01
:100FE000C16E01010451030A08E0010A04E0030A8A
:100FF00006E1C18804D0C18A02D0300EC112010EB0
:10100000C26E1BD003C1DFFFDF50040802E2030EF3
:10101000DF26DF50040DF3500109C26E280EE66E84
:10102000E66A37EC21F0E552E55207D0C282C2B23F
:10103000FED7C3CF03F1C4CF04F10101100E006F3E
:10104000E552E552E7CFD9FF1200D9CFE6FFE1CF55
:10105000D9FF0B0EE12601010251050A63E0060AE1
:1010600007E0010A01E1AAD1030A01E1A7D1A6D153
:1010700092880351080A20E00F0A1CE0010A18E0D8
:10108000030A14E0010A10E0070A0CE0010A08E074
:10109000030A04E0010A12E1200E0FD0210E0DD048
:1010A000220E0BD0230E09D0240E07D0250E05D01A
:1010B000260E03D0270E01D0280ED56ED76AD66A29
:1010C000F294D58E0451030A10E0010A08E0030AE5
:1010D00004E0010A1FE10A0E03D0010E01D00A0E3E
:1010E000E66EE66A93EC21F013D0630EE66EE66AD4
:1010F00093EC21F0E552E552E668030EE66E37EC1C
:1011000021F0E552E5520C0EE66EE66A37EC21F06E
:10111000E552E552D59ED6CF03F1D7CF04F1F2A424
:101120004DD14AD19288270ED56ED76AD66AF294ED
:10113000D58E010EE66EE66A93EC21F0E552E5529B
:10114000D59E080ED6CFDBFFDB50106E116A11342E
:1011500008E210509C08000E115403E2260ED56ED2
:1011600048D0080EDB50106E116A113409E210509D
:101170009C08000E115404E2260ED56E800E33D06A
:10118000080EDB504E0804E2250ED56E400E2BD023
:10119000080EDB50270804E2240ED56E200E23D063
:1011A000080EDB50130804E2230ED56E100E1BD080
:1011B000080EDB50090804E2220ED56E080E13D08B
:1011C000080EDB50040804E2210ED56E040E0BD08D
:1011D000080EDB50020804E2200ED56E020E03D08A
:1011E000280ED56E010EF36E090EF3CFDBFF0A0E4B
:1011F000DB6AD76AD66AF294D58E630EE66EE66A2B
:1012000093EC21F0E552E552E668030EE66E37EC0A
:1012100021F0E552E5520C0EE66EE66A37EC21F05D
:10122000E552E552D59E040ED6CFDBFF050EDB6AF4
:10123000060EDB6A070EDB6A000ED7CFDFFF010E5A
:10124000DB6A020EDB6A030EDB6AD9CFE9FFDACF75
:10125000EAFFEF50EE6AEFCFF4FFEE6EEF50F4CFFF
:10126000EEFFEF6ED9CFE9FFDACFEAFF040EDB50D5
:10127000EE26050EDB50EE22060EDB50EE22070EA8
:10128000DB50EE22D9CFE9FFDACFEAFF0A0E096E72
:101290000A6A0B6A0C6AEECF04F0EECF05F0EECFCF
:1012A00006F0EFCF07F0B0EC27F003C0EDFF02C06F
:1012B000EDFF01C0EDFF00C0EFFF090EDBCF10F026
:1012C0000A0EDBCF11F0126A136AD9CFE9FFDACF29
:1012D000EAFF10C009F011C00AF012C00BF013C0F1
:1012E0000CF0EECF04F0EECF05F0EECF06F0EFCF2E
:1012F00007F0B0EC27F003C0EDFF02C0EDFF01C026
:10130000EDFF00C0EFFFD9CFE9FFDACFEAFFEECF64
:1013100010F010500101036F106A1168126A136A0D
:10132000D9CFE9FFDACFEAFFEE501016EE501116D2
:10133000EE501216EE501316080ED89013321232D9
:1013400011321032E806F9E110C004F1106A116A96
:101350001268136AD9CFE9FFDACFEAFFEE50101610
:10136000EE501116EE501216EE501316100ED890C5
:101370001332123211321032E806F9E110C005F1D1
:10138000106A116A126A1368D9CFE9FFDACFEAFF4F
:10139000EE501016EE501116EE501216EE501316B7
:1013A000180ED8901332123211321032E806F9E1D9
:1013B00010C006F1F2A402D0010101690101100E72
:1013C000006FF56E0B0EE15C02E2E16AE552E16E40
:1013D000F550E552E7CFD9FF1200D9CFE6FFE1CFB4
:1013E000D9FF030EE1263C0EDF6E01010251070A10
:1013F00001E109D1010A01E103D1030A01E19CD015
:10140000010A01E17AD0070A4CE0010A42E0030A2E
:101410000DE0010A01E0F9D04F0EAB16AC9ACF0EE9
:101420009D16C00E0101CF13D76BEFD00F0E031521
:10143000040A14E0070A0CE0010A08E0030A04E0C9
:10144000010A17E19B0E05D0190E03D0330E01D00F
:101450009B0EE66EE66ADFCFE6FF06D04D0EE66E27
:10146000E66AEF0EDF14E66E73EC27F0E552E55204
:10147000E552010103BF03D0CF0EB81402D0300EE5
:10148000B810B86E3F0E0101CF17D86B010ED76FA1
:10149000BCD0ACA2FED703C1E6FFFFEC29F0E552B9
:1014A000B4D00101D85126E0AAC103F1010EDB6AD4
:1014B000D851F36E010EDBCFF4FFF350F45C16E26B
:1014C000010EDB28EA6AAA0FE96E010EEA22EF504C
:1014D000E66E010EDB50EA6AAA0FE96E010EEA22FF
:1014E000E552E750EF6E010EDB2AE2D7D807010183
:1014F000016B8BD00101016988D0DE52030EDD6ED5
:10150000030E01010325F36E010EDBCFF4FFF35050
:10151000F45C01E37AD0ACA2FED7010EDB50EA6A9C
:10152000010FE96E010EEA22EF50E66EFFEC29F0A2
:10153000E552010EDB2AE4D70101D8515EE0020E2C
:1015400003C1DBFFDB500D0805E20D0EF36E020E4A
:10155000F3CFDBFF020EDBCF10F0D851D880105450
:1015600003E2020ED8C1DBFF010EDB6AD851F36E35
:10157000010EDBCFF4FFF350F45C38E2020EDB50D7
:10158000F36E010EDBCFF4FFF350F45C14E2010EB6
:10159000DB50EA6AAA0FE96E010EEA22EF50E66E0E
:1015A000010EDB50030FEA6A010FE96E010EEA2219
:1015B000E552E750EF6E020EDBCFE6FF010EDB5087
:1015C000E552E724EA6AAA0FE96E010EEA22EF501B
:1015D000E66E010EDB50EA6AAA0FE96E010EEA22FE
:1015E000E552E750EF6E010EDB2AC0D7020EDB504A
:1015F000D85F020EDBCF03F108D00101036B05D0E9
:10160000D8C103F102D00101D86B0101100E006FA7
:10161000F56E030EE15C02E2E16AE552E16EF5501F
:10162000E552E7CFD9FF12000101D851106E116ABF
:10163000200E105C000E115801E312009EAA0ED07D
:101640009CEC28F0E66E0101D851D82BEA6AAA0F6B
:10165000E96E010EEA22E552E750EF6E000169A73C
:1016600002D0AB98AB881200D9CFE6FFE1CFD9FF0B
:10167000E652DF6A0A0EDF5C02E3000E01D0010EC3
:10168000106E9E50080B080A01E0010E101409E0CC
:10169000640EE66EE66A37EC21F0E552E552DF2A89
:1016A000E9D70A0EDF5C02E3FF0E02D09E96000E21
:1016B000E552E552E7CFD9FF12009E96C58034EF80
:1016C0000BF0C5841200D9CFE6FFE1CFD9FFFE0EA3
:1016D000DBCFE6FFD0EC29F0E552C750040B01E068
:1016E000010E106E1F0EC5141010F7E1E552E7CF82
:1016F000D9FF1200D9CFE6FFE1CFD9FFFD0EDBCF36
:10170000F3FFDB06F35000091FE06EEC2AF0E66EF3
:10171000FE0EDB50EA6A010FE96E010EEA22E55285
:10172000E750EF6EFE0EDB2AC5B6FED7A1A602D0AB
:10173000FF0E0BD0FD0EDB5002E0C59A01D0C58A2A
:10174000C588C5A8DBD7FDD7000EE552E7CFD9FF86
:101750001200D9CFE6FFE1CFD9FFFD0EDBCFF3FFBB
:10176000DB06F350000937E0C6A61ED0FE0EDB50A4
:10177000EA6A010FE96E010EEA22EF50E66ED0EC44
:1017800029F0E552000902E0FD0E26D0FE0EDB2A0C
:10179000C750040B01E0010E106E1F0EC51410108F
:1017A000F7E1C5ACDAD715D09E96FE0EDB50EA6A9B
:1017B000010FE96E010EEA22EF50C96EFE0EDB2A20
:1017C000C6889EA6FED7C750040BC7E1C750010BC1
:1017D000C4E1FE0E01D0000EE552E7CFD9FF1200A2
:1017E000D9CFE6FFE1CFD9FF020EE1260101025178
:1017F000150A01E193D0010A01E17CD0070A69E0F2
:10180000010A56E0170A48E0010A3BE0070A32E005
:10181000010A27E0030A08E0010A01E096D0C69A0F
:10182000030E0101CE1391D03F0EC716C66AC56ADA
:10183000C68693829380C68A770EC86E0451020AC8
:1018400009E0030A05E0010A08E1C78E770E04D01B
:101850001D0E02D0C78E0B0EC86EFC0E0101CE17F6
:1018600074D02BDF01010351E824E66E2CDFE55232
:10187000010E4FD022DF01010351E8240109E66E79
:1018800033D01BDF010E04C1DBFF01010351E8244B
:10189000046F010EDB283DD010DF01010351E82465
:1018A0000109E66E10DFE55204C1E6FF040E46D0E2
:1018B00004DF030E01010315E824F009E66E03DFDF
:1018C000E55204C1E6FFFFDEE552010EE66E040EAE
:1018D00022D0F3DE030E01010315E824F109E66EC0
:1018E000F2DEE55204C1E6FFEEDEE552010EE66EE1
:1018F000020E24D0E2DE010E05C1DBFF04C105F1BA
:10190000030E01010315E824F009046F010EDB50FA
:10191000020FE66E030EE66E1CDF12D0CEDE030E63
:1019200001010315E824F109E66ECDDEE55204C19C
:10193000E6FFC9DEE55205C1E6FF050EE66EDADE1A
:10194000E552E5520101016FBCDE0101100E006F8E
:10195000F56E020EE15C02E2E16AE552E16EF550DD
:10196000E552E7CFD9FF1200D9CFE6FFE1CFD9FF8B
:10197000E652DF6AFE0EDB500F0B060A14E0030A84
:1019800010E0010A0CE0070A08E0010A04E0030A7B
:101990000CE1040E09D0080E07D0100E05D0200E61
:1019A00003D0400E01D0800EDF6EDF50E552E552CD
:1019B000E7CFD9FF1200D9CFE6FFE1CFD9FFFE0E66
:1019C000DBCFE6FFD1DFE552E81C8A16E552E7CF10
:1019D000D9FF1200D9CFE6FFE1CFD9FFFE0EDBCF52
:1019E000E6FFC2DFE5528A12E552E7CFD9FF1200C7
:1019F000D9CFE6FFE1CFD9FF050EE1260101025163
:101A0000040A01E1B9D0070A01E1ABD0010A01E102
:101A100095D0030A0FE0010A01E0E5D0C69A030E53
:101A20000101CE13CF8FD25101E0CD8BD351CE1314
:101A3000D36BD9D00101D36B020EDF6E010EDB6ACE
:101A4000800EF36E020EF3CFDBFFD26B0101035168
:101A5000060A19E0030A14E0010A0FE0070A0AE087
:101A6000010A05E0030A12E10101040E0ED0010192
:101A70000C0E0BD001011C0E08D001013C0E05D04C
:101A800001017C0E02D00101FC0ED36F0101045153
:101A9000060A14E0030A0CE0060A08E0010A04E062
:101AA000030A0EE1DF6A0CD0010E09D0020E07D046
:101AB000040EDF6E0101010ED26F02D0050EDF6E43
:101AC00001010551040A0FE0070A0AE0010A05E0D6
:101AD000030A0CE1010EDB6A09D0DE52010E05D0CB
:101AE000DE52020E02D0DE52030EDD6E0651020AF5
:101AF00008E0030A08E1800EF36E020EF3CFDBFF6D
:101B000002D0020EDB6A020EDBCFE6FF010EDBCF56
:101B1000E6FFDFCFE6FFE8EC27F0E552E552E552BD
:101B2000FC0E0101CE17CF9FD25101E0CD9BD31DFA
:101B3000CE17D31D9316D3518A1255D003C1E6FF99
:101B40003ADFE5529E9604C1C9FFC6AE03D001013B
:101B5000046904D09EA6FED70101046B03BD43D0E7
:101B60003ED003C1E6FF27DFE55269EC2AF0010110
:101B7000046F03BD38D033D0030E04C1DBFF046B08
:101B8000040EDB6E030EDB50040FF36E040EDBCF8E
:101B9000F4FFF350F45C20E203C1E6FF0CDFE552F2
:101BA0009E96040EDB50EA6A010FE96E010EEA22EE
:101BB000EF50C96EC6AE03D00101046902D09EA6E3
:101BC000FED7800E0101035D04E303C1E6FF02DFDF
:101BD000E552040EDB2AD6D7010103BD04D003C1B0
:101BE000E6FFF8DEE5520101100E006FF56E050EFE
:101BF000E15C02E2E16AE552E16EF550E552E7CFC1
:101C0000D9FF1200D9CFE6FFE1CFD9FF020EE126BE
:101C100001010251030A30E0010A23E0030A08E04F
:101C2000010A39E1C69A030E0101CE13CF8F33D0DA
:101C30000351030A0CE0010A08E0030A04E0010A68
:101C40000BE1120E05D0100E03D0110E01D0120EB2
:101C5000E66EA0EC29F0E552FC0E0101CE17CF9FF5
:101C60001AD003C1E6FF87EC29F0E5520101040513
:101C700012E181B010D0FDD703C1DFFF010E04C116
:101C8000DBFFDBCFE6FFDFCFE6FFF9EC28F0E55224
:101C9000E5520101036F0101100E006FF56E020E97
:101CA000E15C02E2E16AE552E16EF550E552E7CF10
:101CB000D9FF1200D9CFE6FFE1CFD9FF040EE1260C
:101CC00001010251020A3FE0010A3DE0020A09E077
:101CD000010A01E0B2D0030E0101CE13800ECF172E
:101CE000ACD0030E03150101D46F100E01010315D2
:101CF000E8380F0B0101D56FC00E01010315C00AB2
:101D00000FE0400A0AE0C00A05E0400A0CE10101C8
:101D10000A0E08D00101640E05D00101E80E02D0C0
:101D20000101100ED66FFC0E0101CE17CF9F9392CA
:101D30009380949ED40501E17DD0030ED45D01E132
:101D400079D08A927AD0030EDF6E01010325DF5C21
:101D50006BE2DF50EA6A010FE96E010EEA22020E21
:101D6000EFCFDBFF030EDB6ADE52800EDD6E010E6D
:101D7000DB5000084EE20101D45103E0030ED45DB4
:101D800002E18A8201D08A92020EDBCFE6FF010EC9
:101D9000DB50E552E71402E08B8E01D08B9ED651CA
:101DA000E66EE66A37EC21F0E552E5520101D50511
:101DB0000BE181A009D0030EDBCFE7FF010EDB5062
:101DC000E712030EE7CFDBFFD45103E0030ED45D2F
:101DD00002E18A9201D08A82D651E66EE66A37EC39
:101DE00021F0E552E5520101D5510BE181A009D066
:101DF000030EDBCFE7FF010EDB50E712030EE7CF48
:101E0000DBFF010EDBCFF3FFF390F342F3CFDBFFF9
:101E1000AED7DF50EA6A010FE96E010EEA22030E27
:101E2000DBCFEFFFDF2A91D70101D40503E0030EDA
:101E3000D45D02E18A8201D08A920101100E006F06
:101E4000F56E040EE15C02E2E16AE552E16EF550E6
:101E5000E552E7CFD9FF120001010151560A04E013
:101E6000030A03E18A8001D08B80640EE66EE66A85
:101E700037EC21F0E552E552120001010151560AFA
:101E800004E0030A03E18A9001D08B90640EE66EB1
:101E9000E66A37EC21F0E552E5521200D9CFE6FFB1
:101EA000E1CFD9FFE652F00E93128A868A94640E2F
:101EB000E66EE66A37EC21F0E552E552CDDF81505F
:101EC000DF6EDBDFC9DFD9DFDF8E010E0009F6E14F
:101ED0000F0E93168A96E552E552E7CFD9FF12000E
:101EE000D9CFE6FFE1CFD9FFFE0EDB50F00B106E2D
:101EF0000F0E8A1410108A6EAFDFBFDFFE0EDB50AC
:101F00000F0B100DF3CF10F00F0E8A14F3108A6E22
:101F1000A3DFB3DFE552E7CFD9FF1200D9CFE6FF49
:101F2000E1CFD9FF8A84FE0EDBCFE6FFD9DFE55291
:101F3000E552E7CFD9FF1200D9CFE6FFE1CFD9FFB5
:101F40008A94FE0EDBCFE6FFCBDFE552E552E7CF0A
:101F5000D9FF1200D9CFE6FFE1CFD9FF8A94FE0E58
:101F6000DBCFE6FFBDDFE552E552E7CFD9FF120038
:101F7000D9CFE6FFE1CFD9FF020EE12601010251E0
:101F8000060A01E100D1030A01E1EAD0010A01E1F8
:101F9000D4D0070A01E1C2D0010A01E1BBD0030A93
:101FA00014E0010A01E019D10151560A07E0030AC1
:101FB00001E013D1FD0E9312010105D09480FC0EB7
:101FC00093120101CF81CE1308D103C1CAF104C11C
:101FD000CBF10101CC6BCA0509E1100ECB5D06E126
:101FE0000101020E036F0101010ECC6F140EE66EAB
:101FF000E66A93EC21F0E552E5523FDF8A988A9A2F
:102000008A9C8A9E8A948A9601010151560A07E0A9
:10201000030A0BE1020E93160101CE1706D0030E40
:10202000931694900101CE17CE918A888A8A640E05
:10203000E66EE66A37EC21F0E552E5520DDF1DDF72
:10204000140EE66EE66A93EC21F0E552E55204DFE9
:1020500014DF640EE66EE66A37EC21F0E552E552D5
:10206000FBDE0BDF640EE66EE66A37EC21F0E5522C
:10207000E5528A988A8A640EE66EE66A37EC21F0A9
:10208000E552E552E9DEF9DE01010351020A0CE0F6
:10209000030A06E0010A0CE1280EE66E5BDFE5525A
:1020A000200EE66E57DFE552280EE66E53DFE5524E
:1020B000640EE66EE66A37EC21F0E552E552080E52
:1020C000E66E48DFE552640EE66EE66A37EC21F014
:1020D000E552E552010EE66E3DDFE5520A0EE66E70
:1020E000E66A93EC21F0E552E552060EE66E32DF29
:1020F000E552640EE66EE66A37EC21F0E552E552F1
:102100000C0EE66E27DFE552640EE66EE66A37ECEB
:1021100021F011D003C1E6FF01DF5ED003C1E6FF6D
:102120000BDFE552040E0101035D57E2030EE66E7C
:10213000E66A93EC21F0E5524FD0030EDF6E030EFA
:1021400001010325DF5C49E2DF50EA6A010FE96E15
:10215000010EEA22EF50E66EE1DEE552DF2AEFD70C
:10216000030EDF6E030E01010325DF5C36E2DF5054
:10217000EA6A010FE96E010EEA22EF50E66EDCDE3C
:10218000E552DF2AEFD70351010804E20101CB51E8
:1021900001010427010E0315400DF3500425E76EDD
:1021A000010EE7CFDBFF0101CC5111E0010E04C1AC
:1021B000DBFF0101045107080AE2380E106E010E20
:1021C000DBCFE7FF1050E726010EE7CFDBFF010E64
:1021D000DB508009E66EB0DEE5520101100E006FA3
:1021E000F56E020EE15C02E2E16AE552E16EF55045
:1021F000E552E7CFD9FF1200D9CFE6FFE1CFD9FFF3
:10220000040EE12601010251020A5CE0030A08E023
:10221000010A01E080D07DEC2AF00101CF857BD05E
:10222000DE52400EDD6EFD0EDF6E0351090A30E016
:10223000010A2AE00F0A24E0010A1EE0030A18E05E
:10224000010A12E0070A0DE0010A08E0030A03E0B0
:10225000010A22E10DD0DE52180E08D0DE52180E0F
:1022600009D0DE52180E0AD0DE523F0EDD6E0AD0C3
:10227000DE523F0EDD6E0AD0DE523F0EDD6E0AD01A
:10228000010EDB68FC0E07D0010EDB68FD0E03D0EB
:10229000010EDB68FE0EDF6E010EE66EE66A4AECAA
:1022A00028F0E552E5527F0EDF14E66E6CEC29F063
:1022B000E552010EDBCFE6FF2CEC2AF0E5520101DE
:1022C000CF9529D00451E66ED950020FE96EDACFCE
:1022D000EAFFE552E750EE6EED6AD950020FE96E63
:1022E000DACFEAFFEE50ED6EEF6A0351106E116A1D
:1022F000D950020FE96EDACFEAFF1050EE121150FA
:10230000ED12020EDBCFE6FF030EDBCFE6FF4AEC59
:1023100028F0E552E5520101100E006FF56E040E33
:10232000E15C02E2E16AE552E16EF550E552E7CF89
:10233000D9FF1200D9CFE6FFE1CFD9FF040EE12685
:1023400001010251020A5CE0030A08E0010A01E00F
:1023500080D07AEC2AF00101CF837BD0DE52400E90
:10236000DD6EFD0EDF6E0351090A30E0010A2AE03E
:102370000F0A24E0010A1EE0030A18E0010A12E035
:10238000070A0DE0010A08E0030A03E0010A22E15E
:102390000DD0DE52180E08D0DE52180E09D0DE52D3
:1023A000180E0AD0DE523F0EDD6E0AD0DE523F0E0E
:1023B000DD6E0AD0DE523F0EDD6E0AD0010EDB6804
:1023C000FC0E07D0010EDB68FD0E03D0010EDB68AA
:1023D000FE0EDF6E010EE66EE66A1BEC28F0E5529B
:1023E000E5527F0EDF14E66E6CEC29F0E552010E2B
:1023F000DBCFE6FF16EC2AF0E5520101CF9329D09E
:102400000451E66ED950020FE96EDACFEAFFE552C9
:10241000E750EE6EED6AD950020FE96EDACFEAFFAF
:10242000EE50ED6EEF6A0351106E116AD950020F33
:10243000E96EDACFEAFF1050EE121150ED12020EE3
:10244000DBCFE6FF030EDBCFE6FF1BEC28F0E55207
:10245000E5520101100E006FF56E040EE15C02E220
:10246000E16AE552E16EF550E552E7CFD9FF12007F
:10247000D9CFE6FFE1CFD9FF050EE12601010251D8
:10248000050A71E0010A1DE0070A13E0010A01E0F4
:10249000B4D0A69EA69CA68403C1A9FF04C1A8FF30
:1024A000550EA76EAA0EA76EA682A1A8FED7A19868
:1024B000A4D0A69EA69C03C1A9FFA680A8CF04F124
:1024C0009CD0040EDF6E0351E66ED950030FE96E07
:1024D000DACFEAFFE552E750EE6EED6A0451106E76
:1024E000116AD950030FE96EDACFEAFF1050EE26D9
:1024F0001150ED220351E66ED950010FE96EDACF8B
:10250000EAFFE552E750EE6EED6A010EDBCF10F008
:10251000020EDBCF11F0030EDBCF12F0040EDBCF87
:1025200013F01250105C1350115867E2A69EA69C3F
:10253000A684010EDB50A96EDF50EA6A010FE96E36
:10254000010EEA22EF50A86E550EA76EAA0EA76ED6
:10255000A682A1A8FED7A198DF2A010EDB2A020ECF
:10256000D4E3DB2AD2D7040EDF6E0351E66ED950D6
:10257000030FE96EDACFEAFFE552E750EE6EED6A3F
:102580000451106E116AD950030FE96EDACFEAFFD9
:102590001050EE261150ED220351E66ED950010F76
:1025A000E96EDACFEAFFE552E750EE6EED6A010E12
:1025B000DBCF10F0020EDBCF11F0030EDBCF12F0F9
:1025C000040EDBCF13F01250105C1350115815E2BB
:1025D000A69EA69C010EDB50A96EA680DF50EA6A7B
:1025E000010FE96E010EEA22A8CFEFFFDF2A010EEC
:1025F000DB2A020EDCE3DB2ADAD70101100E006FC2
:10260000F56E050EE15C02E2E16AE552E16EF5501D
:10261000E552E7CFD9FF1200D9CFE6FFE1CFD9FFCE
:10262000E652FE0EDB50100DF3CFE9FFF4CFEAFFC8
:10263000410EE926010EEA22EFCFDFFFFE0EDB504E
:10264000100DF3CFE9FFF4CFEAFF410EE926010EAA
:10265000EA22020EE926000EEA22EF50800B02E089
:10266000000EDF80070EDF14070A1CE0010A18E0E5
:10267000030A14E0010A10E0070A0CE0010A08E06E
:10268000030A04E0010A0FE1350E0DD0210E0BD034
:10269000390E09D0180E07D03A0E05D0220E03D0FD
:1026A000360E01D0140EE552E552E7CFD9FF1200E5
:1026B000D9CFE6FFE1CFD9FFFE0EDB50100DF3CFEF
:1026C000E9FFF4CFEAFF410EE926010EEA22080EE7
:1026D000E926000EEA220A0EEF6EFE0EDB50100D08
:1026E000F3CFE9FFF4CFEAFF410EE926010EEA221B
:1026F000080EE926000EEA22010EE926000EEA2263
:10270000080EEF6EFE0EDB50100DF3CFE9FFF4CF95
:10271000EAFF410EE926010EEA22080EE926000E24
:10272000EA22020EE926000EEA22070EEF6EFE0EE6
:10273000DB50100DF3CFE9FFF4CFEAFF410EE9269D
:10274000010EEA22080EE926000EEA22030EE9260F
:10275000000EEA22060EEF6EFE0EDB50100DF3CFD8
:10276000E9FFF4CFEAFF410EE926010EEA22080E46
:10277000E926000EEA22040EE926000EEA22050EE2
:10278000EF6EFE0EDB50100DF3CFE9FFF4CFEAFF42
:10279000410EE926010EEA22080EE926000EEA2281
:1027A000050EE926000EEA22040EEF6EFE0EDB5047
:1027B000100DF3CFE9FFF4CFEAFF410EE926010E39
:1027C000EA22080EE926000EEA22060EE926000E8D
:1027D000EA22030EEF6EFE0EDB50100DF3CFE9FF81
:1027E000F4CFEAFF410EE926010EEA22080EE9269F
:1027F000000EEA22070EE926000EEA22020EEF6E14
:10280000E552E7CFD9FF1200D9CFE6FFE1CFD9FFDC
:10281000FD0EDB50040A20E0070A15E0010A08E07B
:10282000030A29E1FE0EDB500F0B106EF00E07D0ED
:10283000FE0EDB500F0B100DF3CF10F00F0E8A14AD
:102840001010816E18D0FE0EDB500F0B106EF00EC4
:1028500089141010806E0FD0FE0EDB50080DF3505F
:10286000400B116EFE0EDB50070B106EB80E8B1472
:1028700010101110826EE552E7CFD9FF1200D9CFA8
:10288000E6FFE1CFD9FF040EE126020EDB6A030E5C
:10289000DB6AFE0EDB50100DF3CFE9FFF4CFEAFF49
:1028A000410EE926010EEA22030EE926000EEA2275
:1028B000EF50DE6EDD6AFE0EDB50100DF3CFE9FF48
:1028C000F4CFEAFF410EE926010EEA22020EE926C4
:1028D000000EEA22EF50200B01E1B5D0FE0EDB50D6
:1028E000100DF3CFE9FFF4CFEAFF410EE926010E08
:1028F000EA22060EE926000EEA22EECF10F0EFCF14
:1029000011F0D890115004E6080E105C000E11581A
:102910002DE2FE0EDB50100DF3CFE9FFF4CFEAFFFE
:10292000410EE926010EEA22080EE926000EEA22EF
:10293000E9CF10F0EACF11F0FE0EDB50100DF3CF0F
:10294000E9FFF4CFEAFF410EE926010EEA22060E66
:10295000E926000EEA221050EE24E76E1150EE2018
:10296000EA6EE7CFE9FF020EEFCFDBFFFE0EDB5092
:10297000100DF3CFE9FFF4CFEAFF410EE926010E77
:10298000EA22040EE926000EEA22EECF10F0EFCF85
:1029900011F0D890115004E6080E105C000E11588A
:1029A0002DE2FE0EDB50100DF3CFE9FFF4CFEAFF6E
:1029B000410EE926010EEA22080EE926000EEA225F
:1029C000E9CF10F0EACF11F0FE0EDB50100DF3CF7F
:1029D000E9FFF4CFEAFF410EE926010EEA22040ED8
:1029E000E926000EEA221050EE24E76E1150EE2088
:1029F000EA6EE7CFE9FF030EEFCFDBFFDECF10F08B
:102A0000DDCF11F0020EDB50000111AE02D0D890E4
:102A100003D0105C000E115804E2020EDB50DE6E93
:102A2000DD6ADECF10F0DDCF11F0030EDB5011AE0A
:102A300002D0D89003D0105C000E115804E2030EAF
:102A4000DB50DE6EDD6AFE0EDB50100DF3CFE9FFCA
:102A5000F4CFEAFF410EE926010EEA22060EE9262E
:102A6000000EEA22EE2AEF22FE0EDB50100DF3CF0D
:102A7000E9FFF4CFEAFF410EE926010EEA22020E39
:102A8000E926000EEA22EF50400B14E0DECF10F0F2
:102A9000DDCF11F0640E1102F3CF11F01002F3CF6D
:102AA00010F0F4501126F3CFE6FF11C0E6FF37EC2B
:102AB00021F006D0DECFE6FFDDCFE6FF93EC21F07C
:102AC000E552E552F56E040EE15C02E2E16AE55280
:102AD000E16EF550E552E7CFD9FF1200D9CFE6FFFE
:102AE000E1CFD9FF01010251040A01E198D2070A9E
:102AF00001E15BD2010A5CE0030A24E0010A02E082
:102B0000B7EF19F0FE0EDB50040A16E0070A0EE0DC
:102B1000010A06E0030A02E0B7EF19F00F0E01D038
:102B2000F00E93120101CE13B7EF19F00F0E9212AF
:102B30000101CD13B7EF19F0470E94120101CF1325
:102B4000B7EF19F0FE0EDBCFE6FFDBCFE9FFEA6A55
:102B5000E9BEEA68040ED890E936EA36E806FBE1F9
:102B6000410EE926010EEA22EF50E66E55DDE552F0
:102B7000E66E4ADEE552E552FE0EDB50040A13E033
:102B8000070A0CE0010A05E0030A01E0F0D3F00EA9
:102B900001D00F0E93160101CE17E9D3F00E921655
:102BA0000101CD17E4D3B80E94160101CF17DFD37E
:102BB000065102E1010E066FFE0EDBCFE9FFEA6A65
:102BC000E9BEEA68040ED890E936EA36E806FBE189
:102BD000410EE926010EEA22EE52010EEF6EFE0EC4
:102BE000DBCFE9FFEA6AE9BEEA68040ED890E9366D
:102BF000EA36E806FBE1410EE926010EEA22020E62
:102C0000E926000EEA2205C1EFFFFE0EDBCFE9FF49
:102C1000EA6AE9BEEA68040ED890E936EA36E806C0
:102C2000FBE1410EE926010EEA22030EE926000E21
:102C3000EA2206C1EFFF01010451E66EFE0EDBCF72
:102C4000E9FFEA6AE9BEEA68040ED890E936EA3696
:102C5000E806FBE1410EE926010EEA22040EE92610
:102C6000000EEA22E552E750EE6EED6AFE0EDBCF73
:102C7000E9FFEA6AE9BEEA68040ED890E936EA3666
:102C8000E806FBE1410EE926010EEA22040EE926E0
:102C9000000EEA22EE50ED6EEF6A01010351106E54
:102CA000116AFE0EDBCFE9FFEA6AE9BEEA68040EAC
:102CB000D890E936EA36E806FBE1410EE926010E36
:102CC000EA22040EE926000EEA221050EE261150E8
:102CD000ED22FE0EDBCFE9FFEA6AE9BEEA68040EE8
:102CE000D890E936EA36E806FBE1410EE926010E06
:102CF000EA22060EE926000EEA22EE6AED6AFE0ED0
:102D0000DBCFE9FFEA6AE9BEEA68040ED890E9364B
:102D1000EA36E806FBE1410EE926010EEA22020E40
:102D2000E926000EEA22EF50020B020811E1FE0E26
:102D3000DBCFE9FFEA6AE9BEEA68040ED890E9361B
:102D4000EA36E806FBE1410EE926010EEA22EF90A1
:102D5000FE0EDBCFE9FFEA6AE9BEEA68040ED8900E
:102D6000E936EA36E806FBE1410EE926010EEA22E1
:102D7000020EE926000EEA22EF50040B040801E0DF
:102D8000F6D2FE0EDBCFE9FFEA6AE9BEEA68040E7E
:102D9000D890E936EA36E806FBE1410EE926010E55
:102DA000EA22040EE926000EEA22EECF10F0EFCF61
:102DB00011F0113401E3ABD010500008000E115493
:102DC00001E3A5D0FE0EDBCFE9FFEA6AE9BEEA68BF
:102DD000040ED890E936EA36E806FBE1410EE92612
:102DE000010EEA22020EE926000EEA22EF50030B42
:102DF000030A43E0010A1EE0030A0FE0010A5FE153
:102E0000FE0EDBCFE9FFEA6AE9BEEA68040ED8905D
:102E1000E936EA36E806FBE12AD0FE0EDBCFE9FF11
:102E2000EA6AE9BEEA68040ED890E936EA36E806AE
:102E3000FBE140D0FE0EDBCFE9FFEA6AE9BEEA68BB
:102E4000040ED890E936EA36E806FBE1410EE926A1
:102E5000010EEA22EF2AFE0EDBCFE9FFEA6AE9BEA5
:102E6000EA68040ED890E936EA36E806FBE1410E3E
:102E7000E926010EEA22EF2A22D0FE0EDBCFE9FF7F
:102E8000EA6AE9BEEA68040ED890E936EA36E8064E
:102E9000FBE1410EE926010EEA22EF06FE0EDBCF32
:102EA000E9FFEA6AE9BEEA68040ED890E936EA3634
:102EB000E806FBE1410EE926010EEA22EF06FE0ECE
:102EC000DBCFE6FFDBCFE6FF0CEC13F0E552E66E5E
:102ED0009BDCE552E552FE0EDBCFE6FFD0DCE5528F
:102EE000FE0EDBCFE9FFEA6AE9BEEA68040ED8907D
:102EF000E936EA36E806FBE1410EE926010EEA2250
:102F0000040EE926000EEA22EE06EF5A3AD7FE0E2C
:102F1000DBCFE9FFEA6AE9BEEA68040ED890E93639
:102F2000EA36E806FBE1410EE926010EEA22EE52FE
:102F3000EF6AFE0EDBCFE9FFEA6AE9BEEA68040E3B
:102F4000D890E936EA36E806FBE1410EE926010EA3
:102F5000EA22020EE926000EEA22EF50080B0808CA
:102F600001E005D2FE0EDBCFE9FFEA6AE9BEEA68BE
:102F7000040ED890E936EA36E806FBE1410EE92670
:102F8000010EEA22030EE926000EEA22EF500A0F94
:102F9000E66EE66A93EC21F0E552E552FE0EDBCFD9
:102FA000E6FFE66A31DCE55248D0FE0EDBCFE9FFF2
:102FB000EA6AE9BEEA68040ED890E936EA36E8061D
:102FC000FBE1410EE926010EEA22040EE926000E7D
:102FD000EA22EECF10F010500101036FFE0EDBCF9E
:102FE000E9FFEA6AE9BEEA68040ED890E936EA36F3
:102FF000E806FBE1410EE926010EEA22040EE9266D
:10300000000EEA22EECF10F0EFCF11F01016FF0EF7
:10301000111611C010F0116A10C004F1A8D10351AB
:10302000030A01E1D8D0010A0AE0020A01E09FD1B7
:10303000FE0EDBCFE6FF58EC13F0E55298D1FE0E02
:10304000DBCFE9FFEA6AE9BEEA68040ED890E93608
:10305000EA36E806FBE1410EE926010EEA22080EF7
:10306000E926000EEA2204C1EFFFFE0EDBCFE9FFE6
:10307000EA6AE9BEEA68040ED890E936EA36E8065C
:10308000FBE1410EE926010EEA22080EE926000EB8
:10309000EA22010EE926000EEA2205C1EFFFFE0E2C
:1030A000DBCFE9FFEA6AE9BEEA68040ED890E936A8
:1030B000EA36E806FBE1410EE926010EEA22080E97
:1030C000E926000EEA22020EE926000EEA2206C1D7
:1030D000EFFFFE0EDBCFE9FFEA6AE9BEEA68040E05
:1030E000D890E936EA36E806FBE1410EE926010E02
:1030F000EA22080EE926000EEA22030EE926000E57
:10310000EA2207C1EFFFFE0EDBCFE9FFEA6AE9BE64
:10311000EA68040ED890E936EA36E806FBE1410E8B
:10312000E926010EEA22080EE926000EEA22040E24
:10313000E926000EEA2208C1EFFFFE0EDBCFE9FF11
:10314000EA6AE9BEEA68040ED890E936EA36E8068B
:10315000FBE1410EE926010EEA22080EE926000EE7
:10316000EA22050EE926000EEA2209C1EFFFFE0E53
:10317000DBCFE9FFEA6AE9BEEA68040ED890E936D7
:10318000EA36E806FBE1410EE926010EEA22080EC6
:10319000E926000EEA22060EE926000EEA220AC1FE
:1031A000EFFFFE0EDBCFE9FFEA6AE9BEEA68040E34
:1031B000D890E936EA36E806FBE1410EE926010E31
:1031C000EA22080EE926000EEA22070EE926000E82
:1031D000EA220BC1EFFFFE0EDBCFE9FFEA6AE9BE90
:1031E000EA68040ED890E936EA36E806FBE1410EBB
:1031F000E926010EEA22080EE926000EEA22EFCFA8
:1032000004F1FE0EDBCFE9FFEA6AE9BEEA68040ECC
:10321000D890E936EA36E806FBE1410EE926010ED0
:10322000EA22080EE926000EEA22010EE926000E27
:10323000EA22EFCF05F1FE0EDBCFE9FFEA6AE9BE35
:10324000EA68040ED890E936EA36E806FBE1410E5A
:10325000E926010EEA22080EE926000EEA22020EF5
:10326000E926000EEA22EFCF06F1FE0EDBCFE9FFE2
:10327000EA6AE9BEEA68040ED890E936EA36E8065A
:10328000FBE1410EE926010EEA22080EE926000EB6
:10329000EA22030EE926000EEA22EFCF07F1FE0E26
:1032A000DBCFE9FFEA6AE9BEEA68040ED890E936A6
:1032B000EA36E806FBE1410EE926010EEA22080E95
:1032C000E926000EEA22040EE926000EEA22EFCFDC
:1032D00008F1FE0EDBCFE9FFEA6AE9BEEA68040EF8
:1032E000D890E936EA36E806FBE1410EE926010E00
:1032F000EA22080EE926000EEA22050EE926000E53
:10330000EA22EFCF09F1FE0EDBCFE9FFEA6AE9BE60
:10331000EA68040ED890E936EA36E806FBE1410E89
:10332000E926010EEA22080EE926000EEA22060E20
:10333000E926000EEA22EFCF0AF1FE0EDBCFE9FF0D
:10334000EA6AE9BEEA68040ED890E936EA36E80689
:10335000FBE1410EE926010EEA22080EE926000EE5
:10336000EA22070EE926000EEA22EFCF0BF1010157
:10337000100E006FE552E7CFD9FF1200D9CFE6FF5C
:10338000E1CFD9FFFE0EDBCFE9FFEA6AE9BEEA68CA
:10339000040ED890E936EA36E806FBE1410EE9264C
:1033A000010EEA22040EE926000EEA22EECF10F00A
:1033B000EFCF11F0113401E3ACD010500008000E33
:1033C000115401E3A6D0FE0EDBCFE9FFEA6AE9BEA5
:1033D000EA68040ED890E936EA36E806FBE1410EC9
:1033E000E926010EEA22020EE926000EEA22EF503B
:1033F000030B030A43E0010A1EE0030A0FE0010A7F
:103400005FE1FE0EDBCFE9FFEA6AE9BEEA68040E7F
:10341000D890E936EA36E806FBE12AD0FE0EDBCF8B
:10342000E9FFEA6AE9BEEA68040ED890E936EA36AE
:10343000E806FBE140D0FE0EDBCFE9FFEA6AE9BE19
:10344000EA68040ED890E936EA36E806FBE1410E58
:10345000E926010EEA22EF2AFE0EDBCFE9FFEA6A37
:10346000E9BEEA68040ED890E936EA36E806FBE1E0
:10347000410EE926010EEA22EF2A22D0FE0EDBCF12
:10348000E9FFEA6AE9BEEA68040ED890E936EA364E
:10349000E806FBE1410EE926010EEA22EF06FE0EE8
:1034A000DBCFE9FFEA6AE9BEEA68040ED890E936A4
:1034B000EA36E806FBE1410EE926010EEA22EF06B4
:1034C000FE0EDBCFE6FFDBCFE6FF0CEC13F0E552A0
:1034D000E66E04EC14F0E552E552FE0EDBCFE6FF9B
:1034E0003FEC14F0E552FE0EDBCFE9FFEA6AE9BEDD
:1034F000EA68040ED890E936EA36E806FBE1410EA8
:10350000E926010EEA22040EE926000EEA22EE0662
:10351000EF5AFE0EDBCFE9FFEA6AE9BEEA68040E65
:10352000D890E936EA36E806FBE1410EE926010EBD
:10353000EA22040EE926000EEA22EECF10F0EFCFC9
:1035400011F0113404E210500008000E11544EE343
:10355000FE0EDBCFE9FFEA6AE9BEEA68040ED89006
:10356000E936EA36E806FBE1410EE926010EEA22D9
:10357000EE52EF6AFE0EDBCFE9FFEA6AE9BEEA68C7
:10358000040ED890E936EA36E806FBE1410EE9265A
:10359000010EEA22020EE926000EEA22EF50080B85
:1035A000080824E1FE0EDBCFE9FFEA6AE9BEEA681B
:1035B000040ED890E936EA36E806FBE1410EE9262A
:1035C000010EEA22030EE926000EEA22EF500A0F4E
:1035D000E66EE66A93EC21F0E552E552FE0EDBCF93
:1035E000E6FFE66A04EC14F0E552E552E552E7CF57
:1035F000D9FF1200D9CFE6FFE1CFD9FF020EE126B5
:1036000001010251030A01E1FED1010A31E0030A7E
:1036100019E0010A01E035D2FE0EDB50040A0DE08C
:10362000070A09E0010A05E0030A01E02AD2030EB5
:1036300005D00C0E03D0300E01D0C00E9312010144
:10364000CE131FD2FE0EDB50040A0DE0070A09E07C
:10365000010A05E0030A01E014D2FC0E05D0F30EC6
:1036600003D0CF0E01D03F0E93160101CE1709D221
:10367000065102E1010E066FFE0EDBCFE9FFEA6A9A
:10368000E9BEEA68050EEA02F3CFEAFFE902F3CFEA
:10369000E9FFF450EA26910EE926010EEA22010E16
:1036A000EF6EFE0EDBCFE9FFEA6AE9BEEA68050EBF
:1036B000EA02F3CFEAFFE902F3CFE9FFF450EA268A
:1036C000910EE926010EEA22EE5205C1EFFFFE0E31
:1036D000DBCFE9FFEA6AE9BEEA68050EEA02F3CF4A
:1036E000EAFFE902F3CFE9FFF450EA26910EE9265A
:1036F000010EEA22020EE926000EEA2206C1EFFFC1
:103700000451E66EFE0EDBCFE9FFEA6AE9BEEA6825
:10371000050EEA02F3CFEAFFE902F3CFE9FFF45026
:10372000EA26910EE926010EEA22030EE926000E92
:10373000EA22E552E750EE6EED6AFE0EDBCFE9FFBE
:10374000EA6AE9BEEA68050EEA02F3CFEAFFE90297
:10375000F3CFE9FFF450EA26910EE926010EEA22A2
:10376000030EE926000EEA22EE50ED6EEF6A0351D9
:10377000106E116AFE0EDBCFE9FFEA6AE9BEEA6865
:10378000050EEA02F3CFEAFFE902F3CFE9FFF450B6
:10379000EA26910EE926010EEA22030EE926000E22
:1037A000EA221050EE261150ED22FE0EDB50040AE4
:1037B00057E0070A3AE0010A1DE0030A6BE1FE0E3A
:1037C000DBCFE9FFEA6AE9BEEA68050EEA02F3CF59
:1037D000EAFFE902F3CFE9FFF450EA26910EE92669
:1037E000010EEA22EE52EF50010B02E08A8252D023
:1037F0008A9250D0FE0EDBCFE9FFEA6AE9BEEA68A2
:10380000050EEA02F3CFEAFFE902F3CFE9FFF45035
:10381000EA26910EE926010EEA22EE52EF50010B44
:1038200002E08A8637D08A9635D0FE0EDBCFE9FFDC
:10383000EA6AE9BEEA68050EEA02F3CFEAFFE902A6
:10384000F3CFE9FFF450EA26910EE926010EEA22B1
:10385000EE52EF50010B02E08A8A1CD08A9A1AD0ED
:10386000FE0EDBCFE9FFEA6AE9BEEA68050EEA026E
:10387000F3CFEAFFE902F3CFE9FFF450EA26910E15
:10388000E926010EEA22EE52EF50010B02E08A8E89
:1038900001D08A9EFE0EDBCFE9FFEA6AE9BEEA6844
:1038A000050EEA02F3CFEAFFE902F3CFE9FFF45095
:1038B000EA26910EE926010EEA22EE52EF50040BA1
:1038C000040801E0DED0FE0EDBCFE9FFEA6AE9BEC4
:1038D000EA68050EEA02F3CFEAFFE902F3CFE9FF57
:1038E000F450EA26910EE926010EEA22030EE9269B
:1038F000000EEA22EECF10F0EFCF11F011346EE29D
:1039000010500008000E115469E2FE0EDB50040A4C
:1039100024E0070A18E0010A0CE0030A27E18A9074
:10392000010EE66EE66A37EC21F0E552E5528A8038
:103930001DD08A94010EE66EE66A37EC21F0E5525E
:10394000E5528A8413D08A98010EE66EE66A37EC57
:1039500021F0E552E5528A8809D08A9C010EE66E74
:10396000E66A37EC21F0E552E5528A8CFE0EDBCF99
:10397000E9FFEA6AE9BEEA68050EEA02F3CFEAFF68
:10398000E902F3CFE9FFF450EA26910EE926010E91
:10399000EA22020EE926000EEA22EF50E66EE66AFF
:1039A00093EC21F0E552E552FE0EDBCFE9FFEA6A27
:1039B000E9BEEA68050EEA02F3CFEAFFE902F3CFB7
:1039C000E9FFF450EA26910EE926010EEA22030EE1
:1039D000E926000EEA22EE06EF5A75D7FE0EDBCF7F
:1039E000E9FFEA6AE9BEEA68050EEA02F3CFEAFFF8
:1039F000E902F3CFE9FFF450EA26910EE926010E21
:103A0000EA22EF6A3ED0FE0EDBCFE9FFEA6AE9BEAA
:103A1000EA68050EEA02F3CFEAFFE902F3CFE9FF15
:103A2000F450EA26910EE926010EEA22030EE92659
:103A3000000EEA22EECF10F01050036FFE0EDBCF27
:103A4000E9FFEA6AE9BEEA68050EEA02F3CFEAFF97
:103A5000E902F3CFE9FFF450EA26910EE926010EC0
:103A6000EA22030EE926000EEA22EECF10F0EFCF95
:103A700011F01016FF0E111611C010F0116A10C0CF
:103A800004F10101100E006FF56E020EE15C02E21E
:103A9000E16AE552E16EF550E552E7CFD9FF120039
:103AA000D9CFE6FFE1CFD9FFFE0EDBCFE9FFEA6A0F
:103AB000E9BEEA68050EEA02F3CFEAFFE902F3CFB6
:103AC000E9FFF450EA26910EE926010EEA22030EE0
:103AD000E926000EEA22EECF10F0EFCF11F01134FC
:103AE00068E210500008000E115463E2FE0EDB5035
:103AF000040A21E0070A16E0010A0BE0030A23E1A9
:103B00008A90010EE66EE66AB2DBE552E5528A80E3
:103B10001AD08A94010EE66EE66AA9DBE552E552F8
:103B20008A8411D08A98010EE66EE66AA0DBE5521F
:103B3000E5528A8808D08A9C010EE66EE66A97DB19
:103B4000E552E5528A8CFE0EDBCFE9FFEA6AE9BE58
:103B5000EA68050EEA02F3CFEAFFE902F3CFE9FFD4
:103B6000F450EA26910EE926010EEA22020EE92619
:103B7000000EEA22EF50E66EE66AD5DBE552E5522A
:103B8000FE0EDBCFE9FFEA6AE9BEEA68050EEA024B
:103B9000F3CFEAFFE902F3CFE9FFF450EA26910EF2
:103BA000E926010EEA22030EE926000EEA22EE06BD
:103BB000EF5AFE0EDBCFE9FFEA6AE9BEEA68050EBE
:103BC000EA02F3CFEAFFE902F3CFE9FFF450EA2675
:103BD000910EE926010EEA22030EE926000EEA22E2
:103BE000EECF10F0EFCF11F0113404E210500008C6
:103BF000000E115414E3FE0EDBCFE9FFEA6AE9BEC2
:103C0000EA68050EEA02F3CFEAFFE902F3CFE9FF23
:103C1000F450EA26910EE926010EEA22EF6AE552F7
:103C2000E7CFD9FF120001010251030A2EE0010A79
:103C30001BE0030A0FE0010A2CE10101DA6BD96BEA
:103C4000320EDB6FDC6FDD6FDE6FDF6FE06FE16F19
:103C5000E26F1FD003C1DAF10101DA5102E1000E77
:103C600001D0010ED96F15D003C1DBF104C1DCF125
:103C700005C1DDF106C1DEF107C1DFF108C1E0F1E8
:103C800009C1E1F10AC1E2F104D003417F0B010156
:103C9000ED6F0101100E006F120001010251030AC5
:103CA0002EE0010A1BE0030A0FE0010A2EE10101E8
:103CB000E46BE36B320EE56FE66FE76FE86FE96F79
:103CC000EA6FEB6FEC6F21D003C1E4F10101E45125
:103CD00002E1000E01D0010EE36F17D003C1E5F140
:103CE00004C1E6F105C1E7F106C1E8F107C1E9F158
:103CF00008C1EAF109C1EBF10AC1ECF106D00351A8
:103D0000E840E8403F0B0101ED6F0101100E006F2C
:103D10001200D9CFE6FFE1CFD9FF020EE126D00E87
:103D2000DE6E070EDD6E0101DAA11BD093908A8052
:103D3000DBC1E6FF78DAE5520101DB51106E116A52
:103D4000D9CFE9FFDACFEAFF1050EE5E1150ED5AFD
:103D5000D9CFE9FFDACFEAFF640EEE5E000EED5A2E
:103D60008A90DAA31BD093928A82DCC1E6FF5BDAE9
:103D7000E5520101DC51106E116AD9CFE9FFDACFAB
:103D8000EAFF1050EE5E1150ED5AD9CFE9FFDACFBD
:103D9000EAFF640EEE5E000EED5A8A92DAA51BD0A1
:103DA00093948A84DDC1E6FF3EDAE5520101DD51DC
:103DB000106E116AD9CFE9FFDACFEAFF1050EE5E3C
:103DC0001150ED5AD9CFE9FFDACFEAFF640EEE5E6B
:103DD000000EED5A8A94DAA71BD093968A86DEC12C
:103DE000E6FF21DAE5520101DE51106E116AD9CFEA
:103DF000E9FFDACFEAFF1050EE5E1150ED5AD9CF4D
:103E0000E9FFDACFEAFF640EEE5E000EED5A8A9605
:103E1000DAA91BD093988A88DFC1E6FF04DAE5525D
:103E20000101DF51106E116AD9CFE9FFDACFEAFF45
:103E30001050EE5E1150ED5AD9CFE9FFDACFEAFF0C
:103E4000640EEE5E000EED5A8A98DAAB1BD0939AA0
:103E50008A8AE0C1E6FFE7D9E5520101E051106E20
:103E6000116AD9CFE9FFDACFEAFF1050EE5E1150A8
:103E7000ED5AD9CFE9FFDACFEAFF640EEE5E000E0D
:103E8000ED5A8A9ADAAD1BD0939C8A8CE1C1E6FF89
:103E9000CAD9E5520101E151106E116AD9CFE9FF8B
:103EA000DACFEAFF1050EE5E1150ED5AD9CFE9FF9C
:103EB000DACFEAFF640EEE5E000EED5A8A9CDAAFAE
:103EC0001BD0939E8A8EE2C1E6FFADD9E552010177
:103ED000E251106E116AD9CFE9FFDACFEAFF105034
:103EE000EE5E1150ED5AD9CFE9FFDACFEAFF640E4A
:103EF000EE5E000EED5A8A9ED9CFE9FFDACFEAFFD7
:103F0000000ED880EE54000EED5414E2DECF10F017
:103F1000DDCF11F00A0E1102F3CF11F01002F3CF32
:103F200010F0F4501126F3CFE6FF11C0E6FF9FD941
:103F3000E552E552F56E020EE15C02E2E16AE552FD
:103F4000E16EF550E552E7CFD9FF1200D9CFE6FF79
:103F5000E1CFD9FF020EE126E20EDE6E040EDD6E29
:103F60000101E4A11BD094908B80E5C1E6FF5BD9F1
:103F7000E5520101E551106E116AD9CFE9FFDACFA0
:103F8000EAFF1050EE5E1150ED5AD9CFE9FFDACFBB
:103F9000EAFF640EEE5E000EED5A8B90E4A31BD098
:103FA00094928B82E6C1E6FF3ED9E5520101E651CB
:103FB000106E116AD9CFE9FFDACFEAFF1050EE5E3A
:103FC0001150ED5AD9CFE9FFDACFEAFF640EEE5E69
:103FD000000EED5A8B92E4A51BD094948B84E7C11C
:103FE000E6FF21D9E5520101E751106E116AD9CFE0
:103FF000E9FFDACFEAFF1050EE5E1150ED5AD9CF4B
:10400000E9FFDACFEAFF640EEE5E000EED5A8B9404
:10401000E4AD1BD0949C8B8CEBC1E6FF04D9E55238
:104020000101EB51106E116AD9CFE9FFDACFEAFF37
:104030001050EE5E1150ED5AD9CFE9FFDACFEAFF0A
:10404000640EEE5E000EED5A8B9CE4AF1BD0949E86
:104050008B8EECC1E6FFE7D8E5520101EC51106E02
:10406000116AD9CFE9FFDACFEAFF1050EE5E1150A6
:10407000ED5AD9CFE9FFDACFEAFF640EEE5E000E0B
:10408000ED5A8B9ED9CFE9FFDACFEAFF000ED88038
:10409000EE54000EED5414E2DECF10F0DDCF11F03F
:1040A0000A0E1102F3CF11F01002F3CF10F0F4500A
:1040B0001126F3CFE6FF11C0E6FFD9D8E552E5524D
:1040C000F56E020EE15C02E2E16AE552E16EF55046
:1040D000E552E7CFD9FF1200D9CFE6FFE1CFD9FFF4
:1040E000020EE12601010251040A33E0070A27E02B
:1040F000010A19E0030A07E0010A32E173EC2AF031
:104100000101CD892DD03F0EE66E50EC29F0E5522D
:10411000000EE66EE66A34EC29F0E552E55292882C
:104120000101CD991DD0DAEC28F0F3CFDEFFF4CFFA
:10413000DDFFDFCF03F1010EDBCF04F111D003C1AE
:10414000DFFF010E04C1DBFFDECFE6FFDDCFE6FFC0
:1041500003D0000EE66EE66A34EC29F0E552E55233
:104160000101100E006FF56E020EE15C02E2E16AE1
:10417000E552E16EF550E552E7CFD9FF1200D9CFF5
:10418000E6FFE1CFD9FF020EE12601010251040A48
:1041900034E0070A28E0010A1AE0030A07E0010AEE
:1041A00033E177EC2AF00101CF812ED0070EE66EC5
:1041B00079EC28F0E552CD96000EE66EE66A18EC32
:1041C00029F0E552E55294800101CF911DD0BBEC5E
:1041D00028F0F3CFDEFFF4CFDDFFDFCF03F1010ED8
:1041E000DBCF04F111D003C1DFFF010E04C1DBFFFF
:1041F000DECFE6FFDDCFE6FF03D0000EE66EE66A17
:1042000018EC29F0E552E5520101100E006FF56E31
:10421000020EE15C02E2E16AE552E16EF550E55220
:10422000E7CFD9FF1200D9CFE6FFE1CFD9FFE652A1
:10423000DF6A0101ED51D880DF5407E30A0EE66E14
:104240005EEC2AF0E552DF2AF4D7DF6AFE0EDB507F
:10425000D880DF5407E30A0EE66E5EEC2AF0E552E2
:10426000DF2AF4D7E552E552E7CFD9FF1200D9CFC4
:10427000E6FFE1CFD9FFE652FF0EE76EFD0EDBCF82
:1042800010F0E7501016116A1050DF6EDF50000872
:1042900005E2DFCFE6FF5EEC2AF0E552FD0EDBCF54
:1042A00010F0FE0EDBCF11F011C010F0116A1050AB
:1042B000DF6EDF50000832E2DFCFE6FF42EC2AF08B
:1042C000E552DFCFE6FF42EC2AF0E552DFCFE6FF12
:1042D00042EC2AF0E552DFCFE6FF5EEC2AF0E55231
:1042E000DFCFE6FF5EEC2AF0E552DFCFE6FF5EECC3
:1042F0002AF0E552DFCFE6FF5EEC2AF0E552DFCF91
:10430000E6FF5EEC2AF0E552DFCFE6FF5EEC2AF036
:10431000E552DFCFE6FF5EEC2AF0E552E552E552CA
:10432000E7CFD9FF1200D9CFE6FFE1CFD9FFE150A7
:10433000FD0FE96EFF0EDA20EA6E000ED880EE5413
:10434000000EED5412E2FD0EDBCFE6FFE8EC29F0A3
:10435000E552FD0EDBCFE6FF42EC2AF0E552FD0E02
:10436000DBCFE6FF42EC2AF0E552E552E7CFD9FF7A
:104370001200D9CFE6FFE1CFD9FF030EE1260101FC
:10438000440E016F3F0E006F040EDF6E0251E66EA9
:10439000D950010FE96EDACFEAFFE552E750EE6E31
:1043A000ED6A010EDBCF10F0020EDBCF11F00251EF
:1043B0000425136AE850105C1350115814E2A69EAD
:1043C000010EDB50A96EA680DF50EA6A010FE96E8C
:1043D000010EEA22A8CFEFFFDF2A010EDB2A020E30
:1043E000E0E3DB2ADED7F56E030EE15C02E2E16A70
:1043F000E552E16EF550E552E7CFD9FF1200D9CF73
:10440000E6FFE1CFD9FF030EE1260101010E006FA7
:10441000450E016F040EDF6E0251E66ED950010F9A
:10442000E96EDACFEAFFE552E750EE6EED6A010E73
:10443000DBCF10F0020EDBCF11F001010251042599
:10444000136AE850105C135011581CE2A69EA68413
:10445000010EDB50A96EDF50EA6A010FE96E010E12
:10446000EA22EF50A86E550EA76EAA0EA76EA6827E
:10447000A1A8FED7A198DF2A010EDB2A020ED7E3FE
:10448000DB2AD5D7F56E030EE15C02E2E16AE55264
:10449000E16EF550E552E7CFD9FF1200C282C2B2F9
:1044A000FED712009494780ECB6E0C0EBD6EBE6ECD
:1044B000040ECA6E12006C500CE1689604010051A3
:1044C0003C0BE842E8420D0802E10AD8010C1ED874
:1044D000010C040E6C5C03E1689627D8010C000CFB
:1044E000D9CFE6FFE1CFD9FFE652040104BF046B48
:1044F0000001686B606B616B666B676B02EC24F0AC
:10450000ECD8E552E552E7CFD9FF1200020E0001C8
:10451000605D09E1A3D8040100BD02D0C80E01D03E
:10452000880E006F1200B2EF23F0040E0101F85D57
:1045300009E11AC46EFF6E50000802E2050E01D0B8
:10454000030EF86F0001600510E111D8020E0001A2
:10455000685D03E10401840E06D0040104BD02D0AD
:10456000C80E01D0880E046F1200B2EF23F0D9CF2D
:10457000E6FFE1CFD9FF020EE1260001080E665DDD
:10458000000E67590DE266C0DEFF67C0DDFF6851AF
:1045900002E1010E03D0680506E1020E686F03D048
:1045A000080EDE6EDD6A040104930491010EDB50F7
:1045B0000413DFCF05F4000EDB500001665F010E2F
:1045C000DB50675B200E646F040E656F0101F9A379
:1045D0001DD0D9CFE9FFDACFEAFFEE50ED1032E07F
:1045E00062C0F6FF63C0F7FF0800F55064C0E9FF42
:1045F00065C0EAFFEF6E0001642B000E6523622B9D
:104600006323DF06010EE5E2DB06E3D7D9CFE9FF3E
:10461000DACFEAFFEE50ED1015E062C0E9FF63C0AB
:10462000EAFFEF5064C0E9FF65C0EAFFEF6E0001EA
:10463000642B000E6523622B6323DF06010EE6E286
:10464000DB06E4D7F56E020EE15C02E2E16AE552B8
:10465000E16EF550E552E7CFD9FF1200D9CFE6FF62
:10466000E1CFD9FF020EE126030E04010015E76E2B
:10467000010EE7CFDBFF01C4DFFFDE50000166273C
:10468000DD506723200E626F040E636FD9CFE9FF00
:10469000DACFEAFFEE50ED1014E062C0E9FF63C02C
:1046A000EAFFEF5064C0E9FF65C0EAFFEF6E642BDC
:1046B000000E6523622B6323DF06010EE7E2DB06B3
:1046C000E5D7F56E020EE15C02E2E16AE552E16EC9
:1046D000F550E552E7CFD9FF12006D980001615106
:1046E0000BE10401080E016F180E026F040E036F38
:1046F000840E006F040123D0040118AF22D0000102
:10470000665104011E5D0001675104011F5904E256
:104710001EC466F01FC467F02ADF0001010E606F3F
:104720000401080E016F180E026F040E036F800E55
:10473000006F0401200E066F040E076FC80E046F91
:1047400012000001020E606F0401056BC80E046FB9
:104750000401080E016F200E026F040E036FC80ED5
:10476000006F1200D9CFE6FFE1CFD9FFE652020E6B
:104770000001605D35E16D50100B32E00401015124
:10478000106E116A080E10182BE1115029E100512A
:104790003C0BE842E8420D0823E10051800B20E188
:1047A000180E026F040E036FDF6ADF50106E116A7D
:1047B000080E105C000E115820E2DF50EA6A200F4C
:1047C000E96E040EEA22EF50E66EDF50EA6A180F37
:1047D000E96E040EEA22E552E750EF6EDF2AE5D7D4
:1047E0000001606B0401080E016F180E026F040EC9
:1047F000036F8C0E006F0401046BE552E552E7CFA6
:10480000D9FF120004011851600BE842E842E84267
:10481000E842E842000901E012001951070A4CE0A1
:104820000B0A4AE0070A3BE0010A27E00B0A23E0F3
:10483000020A21E0030A1DE0080A12E0010A0EE064
:104840000F0A0AE0030A01E012000001010E616F85
:104850000101040EF86F12005DEF24F0B4EF24F0B4
:104860000001010E616F0001FA0E626F010E636FAD
:1048700010D0DBEF24F026EF25F00001010E616F70
:1048800004011C510001626F636BFB0E6227010E75
:1048900063230101F9930001010E666F120000010C
:1048A000010E616F04011C51EA6AFB0FE96E010EF3
:1048B000EA221AC4EFFF12001200800E0401185DF4
:1048C00052E11B51030A30E0010A0CE0030A49E1FE
:1048D0000001010E616F0001A80E626F4D0E636F43
:1048E000120E3CD00001010E616F04011A51F66EE8
:1048F000F76AD890F636F7363E0EF6264E0EF722B9
:104900000900F5CF62F00A00F5CF63F0020E000156
:10491000F76A6225F66E6351F7220900F5CF66F05B
:104920000A00F5CF67F01DD00001010E616F040190
:104930001A51F66EF76AD890F636F736420EF6261A
:104940004E0EF7220900F5CF62F00A00F5CF63F0B2
:1049500062C0F6FF63C0F7FF0800F5500001666F04
:10496000676B0101F98312000001010E616F0F0EE8
:10497000E66E710EE66E0F0EE66E31EC26F0E55235
:10498000E552E552010EE66EFB0EE66E010EE66E96
:1049900031EC26F0E552E552E5521AC4FAF1040171
:1049A0001A5104E10101050EF86F12000101060E13
:1049B000F86F46EF26F00401206B216B04011851BB
:1049C0001F0B020A13E0030A0DE0010A31E10001A6
:1049D000010E616F040120810101F9A129D00401B8
:1049E000208326D00001010E616F22D00001010E4C
:1049F000616F04011C510F0B080DF350116A000F79
:104A0000106E040E11221C51800B01E0010E040DEA
:104A1000F35000011024646F000E1120656F64C014
:104A2000E9FFEA6EEF50040B03E00401010E206F72
:104A3000000161050AE10001200E626F040E636F40
:104A40000101F9930001020E666F120004011A05BC
:104A500010E118511F0B00090CE10001010E616FFC
:104A6000030E0401195D03E10101F98102D0010186
:104A7000F99104011A5136E118511F0B020832E175
:104A80001C510F0B00092EE00001010E616F0401A3
:104A90001C510F0B080DF350116A000F106E040E1D
:104AA00011221C51800B01E0010E040DF350000196
:104AB0001024646F000E1120656F030E0401195D50
:104AC00002E1840E03D01CAF07D0400E64C0E9FFA2
:104AD00065C0EAFFEF6E1200880E64C0E9FF65C092
:104AE000EAFFEF6E12006DA60CD80101F80508E18F
:104AF0006DBA06D0686A696A69806988020EF86FC3
:104B000012006D6A696A6D860101010EF86F12006C
:104B10006D6A696A0101F86B120088EF25F00101E6
:104B2000F85101E112006850040B04E06950040BD5
:104B300001E042D86DB212006850010B04E06950E8
:104B4000010B01E066D86850100B04E06950100BAF
:104B500001E02ED86850400B04E06950400B01E0A2
:104B600044D86850200B04E06950200B01E03FD886
:104B70006850020B04E06950020B01E048D8030EB4
:104B80000101F85D01E212000101FC6B040EFC5D05
:104B90000EE26850080B0BE06950080B08E05BEC74
:104BA00022F0000901E168960101FC2BEFD7120009
:104BB000698468986D8212006D92699468A402D02D
:104BC0006894FCD712000101F9A10ED06D926D849A
:104BD0000101080EFD6F070EFE6FFD07000EFE5B64
:104BE000FD51FE11FAE16D941200689C120070A054
:104BF0000CD0800E0401005D07E1840E0401045D09
:104C000003E104018C0E006F7090689A12006A6ACA
:104C100012006A6A686A9F0E6B6E7B0E696E6E6A1E
:104C20000F0EE66E710EE66E0F0EE66E1AD8E552A6
:104C3000E552E552160E706E68A608D06896000020
:104C400000000000000000000000F6D76D98B2ECF4
:104C500023F00101F9910101FA6B0101030EF86FD4
:104C60001200D9CFE6FFE1CFD9FFFD0EDBCFE9FF80
:104C7000FE0EDBCFEAFFFC0EDB5004E0EE6AFC0E1A
:104C8000DB06F9D7E552E7CFD9FF12000101FF6B30
:104C90001E0E716E0401400E096F280E0A6F040E7D
:104CA0000B6F880E086F0401680E0E6F040E0F6FF5
:104CB000400E0C6F1200D9CFE6FFE1CFD9FFE652CC
:104CC000FC0EDB50400805E2400EF36EFC0EF3CF05
:104CD000DBFFDF6AFC0EDB50DF5C19E2DF50E76EC2
:104CE000FD0EDBCFE9FFFE0EDBCFEAFFE750E92642
:104CF000000EEA22EF50E66EDF50EA6A680FE96EB6
:104D0000040EEA22E552E750EF6EDF2AE3D7FC0EED
:104D1000DBCF0DF4400E04010C170C7D880E0C1334
:104D2000E552E552E7CFD9FF1200D9CFE6FFE1CF38
:104D3000D9FF0101FF6B040108BF30D0FC0EDBCFAF
:104D400010F00951D880105403E2FC0E09C4DBFFB7
:104D50000101FF6BFC0EDB50FF5D19E2FF51EA6AB7
:104D6000280FE96E040EEA22EF50E66EFF51E76E5F
:104D7000FD0EDBCFE9FFFE0EDBCFEAFFE750E926B1
:104D8000000EEA22E552E750EF6EFF2BE3D7040155
:104D9000400E096F0817087D880E08130101FF51A6
:104DA000E552E7CFD9FF120012010002000000080F
:104DB000D8040BFF010001020001090220000101DB
:104DC00000C03209040000020000000007050102D3
:104DD00040000007058102400000040309042A0383
:104DE00073007000720075007400200028007700C6
:104DF000770077002E007300700072007500740059
:104E00002E0064006500290036035500530042005F
:104E1000340061006C006C002D004D004300440024
:104E2000310030002000280073007000720075000F
:104E30007400200032003000310032002900BA4DE9
:104E4000BA4DDA4DDE4D084E2A0EF66E080EF76E9C
:104E5000000EF86E01010900F550F36F0900F550DE
:104E6000F46F03E1F36701D03DD00900F550EE6F18
:104E70000900F550EF6F0900F550F06F09000900C7
:104E8000F550E96E0900F550EA6E090009000900C5
:104E9000F550F16F0900F550F26F09000900F6CFE7
:104EA000F5F1F7CFF6F1F8CFF7F1EEC1F6FFEFC16C
:104EB000F7FFF0C1F8FF0101F15302E1F25307E0FF
:104EC0000900F550EE6EF107F8E2F207F9D7F5C1E7
:104ED000F6FFF6C1F7FFF7C1F8FF0101F307000E77
:104EE000F45BBFD71200D9CFE6FFDACFE6FFE1CF00
:104EF000D9FFE2CFDAFFAC6AAB6AFD0EDBB0AC885B
:104F0000DBA202D0AC8CAB8CDBB4AC8EDBA602D0C7
:104F1000AB8801D0AB8ADBA802D0AC8401D0AC94C2
:104F20009E98DBAC02D09D8A01D09D9A9E9ADBAE02
:104F300002D09D8801D09D98FB0EDB50AF6EFB0E1A
:104F4000FC0EDBCF11F011C010F0116A1050B06EE2
:104F5000AC8AAB8EE552E5CFDAFFE7CFD9FF12007E
:104F600004500902F3CF00F0F4CF01F00A02F3502D
:104F70000126000EF420026E04500B02F3500226AC
:104F8000000EF420036E04500C02F350032605506B
:104F90000902F3500126F4500222000E03220550AC
:104FA0000A02F3500226F450032205500B02F3507C
:104FB000032606500902F3500226F450032206503D
:104FC0000A02F350032607500902F3500326120089
:104FD000D9CFE6FFDACFE6FFE1CFD9FFE2CFDAFFA4
:104FE0003F0EC716C66AFD0EDB50C612FB0EDB5025
:104FF000C712FC0EDB50030A09E0010A04E0020AB2
:1050000006E1C78C04D0C78CC68801D0C688FD0EC7
:10501000DB50050A03E0010A04E1928A9382C79EED
:1050200001D09392949E9380C68AE552E5CFDAFF31
:10503000E7CFD9FF1200D9CFE6FFDACFE6FFE1CF05
:10504000D9FFE2CFDAFFE652E652FC0EDBCF10F0DA
:10505000FD0EDBCF11F0060ED89010361136E804A5
:10506000FBE110C0DEFF11C0DDFF010EDB50BB6EA7
:10507000DF50E840E8403F0B300B106ECF0EBA1403
:105080001010BA6EE552E552E552E5CFDAFFE7CFF0
:10509000D9FF1200D9CFE6FFDACFE6FFE1CFD9FF83
:1050A000E2CFDAFFE652E652FC0EDBCF10F0FD0E47
:1050B000DBCF11F0060ED89010361136E804FBE174
:1050C00010C0DEFF11C0DDFF010EDB50BE6EDF50F1
:1050D000E840E8403F0B300B106ECF0EBD141010AF
:1050E000BD6EE552E552E552E5CFDAFFE7CFD9FFD5
:1050F0001200D9CFE6FFDACFE6FFE1CFD9FFE2CF4A
:10510000DAFFFD0EDB507E0BB16EB36AB26AA1927C
:10511000FD0EDBAE02D0A08201D0A092DBB2CD8624
:10512000DBA002D0B18E01D0B19EB180E552E5CFB7
:10513000DAFFE7CFD9FF1200D9CFE6FFDACFE6FFDB
:10514000E1CFD9FFE2CFDAFFE652F20E0001691794
:10515000ABAC03D06991ABB06981ABB46985ABB23C
:105160006987AE50DF6EDF50E552E552E5CFDAFFDA
:10517000E7CFD9FF1200D9CFE6FFDACFE6FFE1CFC4
:10518000D9FFE2CFDAFFE652E652B250DF6E010EEF
:10519000B3CFDBFFDECF10F0DDCF11F010C0F3FF97
:1051A00011C0F4FFE552E552E552E5CFDAFFE7CF53
:1051B000D9FF1200D9CFE6FFDACFE6FFE1CFD9FF62
:1051C000E2CFDAFFE652E652D650DF6E010ED7CFBD
:1051D000DBFFDECF10F0DDCF11F010C0F3FF11C008
:1051E000F4FFE552E552E552E5CFDAFFE7CFD9FF0C
:1051F0001200D9CFE6FFDACFE6FFE1CFD9FFE2CF49
:10520000DAFFC688FD0EDB50C96EC7A0FED7FC0EC4
:10521000DB50C96EC7A0FED7C698C96AC7A0FED723
:10522000C688C950E552E5CFDAFFE7CFD9FF1200B3
:10523000D9CFE6FFDACFE6FFE1CFD9FFE2CFDAFF41
:10524000E652E652FC0EDBCFDEFFDBCFDDFF010EC8
:10525000DB50B36EDF50B26EE552E552E552E5CF5A
:10526000DAFFE7CFD9FF1200D9CFE6FFDACFE6FFAA
:10527000E1CFD9FFE2CFDAFFE652E652FC0EDBCFF8
:10528000DEFFDBCFDDFF010EDB50D76EDF50D66EC9
:10529000E552E552E552E5CFDAFFE7CFD9FF12003C
:1052A000D9CFE6FFDACFE6FFE1CFD9FFE2CFDAFFD1
:1052B000FD0EDB507F0BD56ED76AD66AF294FD0ED9
:1052C000DBAE02D0F28A01D0F29AD58EE552E5CF5C
:1052D000DAFFE7CFD9FF1200D9CFE6FFDACFE6FF3A
:1052E000E1CFD9FFE2CFDAFFFD0EDB50FB0BCA6E38
:1052F000CC6A9E92FD0EDBAE02D09D8201D09D92C3
:10530000CA84E552E5CFDAFFE7CFD9FF1200D9CF43
:10531000E6FFDACFE6FFE1CFD9FFE2CFDAFFC688BA
:10532000FD0EDB50C96EC6AE02D0FF0E03D0C7A083
:10533000FED7000EE552E5CFDAFFE7CFD9FF120026
:10534000D9CFE6FFDACFE6FFE1CFD9FFE2CFDAFF30
:105350003F0EC716C66AFD0EDB50C612949E93928E
:105360009380C68AE552E5CFDAFFE7CFD9FF120076
:1053700004D80FD820EC05F0FCD70F0EC112140E84
:105380006F6E0101F86B0101F96B0101FA6B1CEF03
:1053900004F073EC25F06FBE02D08FEC25F0120004
:1053A000D9CFE6FFDACFE6FFE1CFD9FFE2CFDAFFD0
:1053B000FD0EDB50C96EC6AE02D0FF0E03D0C7B0E3
:1053C000FED7000EE552E5CFDAFFE7CFD9FF120096
:1053D000FF0EE350156EEF0E01D0F30EE76EE72ED1
:1053E000EFEF29F00C0E146EE76AE72EF5EF29F0C7
:1053F000142EF4EF29F0152EEDEF29F01200D9CF7D
:10540000E6FFDACFE6FFE1CFD9FFE2CFDAFFACACBF
:1054100004D0AC90000169B3AC80FD0EDB50AD6EE2
:10542000E552E5CFDAFFE7CFD9FF1200D9CFE6FF8B
:10543000DACFE6FFE1CFD9FFE2CFDAFF0C0EBA6E8A
:10544000CA949492FD0EDB50CB6ECA84E552E5CF30
:10545000DAFFE7CFD9FF1200D9CFE6FFDACFE6FFB8
:10546000E1CFD9FFE2CFDAFF0C0EBD6ECA94FD0E7C
:10547000DB50CB6E9494CA84E552E5CFDAFFE7CFD8
:10548000D9FF1200FF0EE350156E480E01D04C0EEE
:10549000E76EE72EFED7E76AE72EFED7152EF7D781
:1054A0000000120013EE00F023EE00F0F86A0F9CEB
:1054B00024EC27F0B8EC29F0FDD71200FF0EE350E2
:1054C000E84E1200000000D000D000D0E82EFAD73D
:1054D0001200C96AC7A0FED7C9501200C586C7A06E
:1054E000FED7C9501200F29A7F0ED56E1200B1900D
:1054F000A0921200BA6A94821200BD6A94841200CB
:105500000210007FFFC700000000000064000000E0
:105510000032323232323232320000323232323201
:1055200032323264FFFFFFFFFFFFFFFFFFFFFFFF8D
:10553000FFFFFFFFFFFFFFFFFFFFFFFFFFFFFFFF7B
:020000040020DA
:080000000F0F0F0F0F0F0F0F80
:020000040030CA
:08000000240E281E00018100FE
:0200000400F00A
:100000001829E5E5011000F502E102E1E5E1F5E579
:10001000E7D912D9E6E1D9E6DF01EDD8DF070AE634
:100020005E2AE5DFF4DFFEDBD8DF070AE65E2AE5BD
:10003000DFF4E5E5E7D912D9E6E1D9E6FFE7FDDB34
:1000400010E7101110DFDF0005DFE65E2AE5FDDBBB
:1000500010FEDB1111101110DFDF0032DFE6422A43
:10006000E5DFE6422AE5DFE6422AE5DFE65E2AE54D
:10007000DFE65E2AE5DFE65E2AE5DFE65E2AE5DF0B
:10008000E65E2AE5DFE65E2AE5DFE65E2AE5E5E5EF
:10009000E7D912D9E6E1D9E1FDE9FFDAEA00D8EEC5
:1000A00000ED12FDDBE6E829E5FDDBE6422AE5FD91
:1000B000DBE6422AE5E5E7D912D9E6E1D903E10119
:1000C00044013F0004DF02E6D901E9DAEAE5E7EEA0
:1000D000ED01DB1002DB11020413E810131114A66A
:1000E00001DBA9A6DFEA01E901EAA8EFDF01DB02F3
:1000F000E0DBDEF503E102E1E5E1F5E5E7D912D960
:00000001FF
